:100000002090047400800274012091047900800221
:1000100079014930E004D2928002C29220930474A4
:10002000008002740120940479008002790149F46F
:1000300030E004D2958002C29520B00474008002A2
:10004000740120B1047900800279015930E004D2B2
:10005000B28002C2B220B30474008002740120B4E2
:100060000479008002790159F430E004D2B58002AD
:10007000C2B5209604740080027401F430E004D20A
:07008000970100C297010087
:00000001FF
